:1000000000308A0036290000831A0A28A500030E52
:10001000A6000F288312A500030EA600A6140A0846
:10002000AD008A018313A50E0408A7002008A800CC
:100030002108A9002208AA002308AB002408AC006C
:1000400083128C308400001C27280C183C282708B9
:1000500084002808A0002908A1002A08A2002B0873
:10006000A3002C08A4002D088A00260E830083120A
:10007000250EA61883160900B30A0319B40ABF088F
:1000800003194E2837080319B803B703B808031D2E
:100090004D283708013C0318BF015E28B70A031931
:1000A000B80A3808023C03185E28FF3A031D5C2892
:1000B0003708FE3C03185E280130BF00C008031952
:1000C0006D2839080319BA03B903BA08031D6C284F
:1000D0003908013C0318C0017D28B90A0319BA0A7E
:1000E0003A08023C03187D28FF3A031D7B28390893
:1000F000FE3C03187D280130C000C10803198C287C
:100100003B080319BC03BB03BC08031D8B283B0839
:10011000013C0318C1019C28BB0A0319BC0A3C0816
:10012000023C03189C28FF3A031D9A283B08FE3C1A
:1001300003189C280130C1000C108A11272845089B
:10014000B2004408B1004308B0004208AF00832960
:100150002030CE00CA01CB01CC01CD014508A3005F
:100160004408A2004308A1004208A0000310201C7C
:10017000C7284608CA0747080318470FCB0748088F
:100180000318480FCC0749080318490FCD07CD0CB9
:10019000CC0CCB0CCA0CA30CA20CA10CA00CCE0B4B
:1001A000B6280929A101A201A001A3014808031D45
:1001B000DC2847080319F6281030C9000310C50DC4
:1001C000C60DA00DA30D48082302031DE92847080A
:1001D0002002031CF2284708A002031CA3034808BE
:1001E000A3020314A10DA20DC90BDE2800003129C2
:1001F0003208C5003108C4003008C3002F08C2000F
:100200004130C900C630C8004E30C7006D30C6004E
:10021000A82839302007AF002108B000303003187B
:100220003130B0072208B100003003180130B107A7
:100230002308B200003003180130B2073108A000D3
:100240003208A100A201A3013208C4003108C30092
:100250003208C6003108C5007F30C800FF30C70033
:10026000D2282008A1002308A200003484011F30F6
:1002700083051F1383161F109F101F119F11073036
:100280008312990083160508831219088C11AE0198
:100290000130AF00B001B101B201831685018312B4
:1002A0008501853090008F018E01BF01C001C10121
:1002B000B601B501B401B301013083169B009C1354
:1002C0001C141A088312BD00BD0A013083169B005E
:1002D00083123D0883169A001C1583120B08A00098
:1002E0008B13831655309D00AA309D009C149C18DA
:1002F00077291C11831220088B04C501C401C30196
:100300003D08C2009F28F820210DB700B80103184E
:10031000B80AB70DFC30B705F820210DB900BA01B5
:100320000318BA0AB90DFC30B905F820210DBB003D
:10033000BC010318BC0ABB0DFC30BB05F82021082A
:100340000739BE00BE08031DA7290730BE0083166B
:100350000C14C03083128B043608033C0318CE29DA
:100360003408263C0318C629FF3A031DBB2933086D
:10037000F53C0318C629B401B301F8202108073958
:10038000BE00BE08031DC6290730BE00B601B50178
:100390008316850183123E088500F529370835024A
:1003A000031DDA2938083602031DDA298316851061
:1003B0008312851039083502031DE6293A083602F2
:1003C000031DE62983160510831205103B0835022C
:1003D000031DF2293C083602031DF229831605117C
:0E03E00083120511B50A0319B60AAC29630091
:02400E00E2319D
:00000001FF
